:020000040801F1
:1000000000000220CD320108C9200108CD200108DE
:10001000D1200108D5200108D920010800000000E6
:10002000000000000000000000000000DD200108CA
:10003000E120010800000000E5200108E920010896
:100040001D3301081D3301081D3301081D3301084C
:100050001D3301081D3301081D3301081D3301083C
:100060001D3301081D3301081D3301081D3301082C
:100070001D3301081D3301081D3301081D3301081C
:100080001D3301081D3301081D3301081D3301080C
:100090001D3301081D3301081D3301081D330108FC
:1000A0001D3301081D3301081D3301081D330108EC
:1000B0001D3301081D3301081D3301081D330108DC
:1000C0001D3301081D3301081D3301081D330108CC
:1000D0001D330108F9200108052101081D3301081D
:1000E0001D3301081D3301081D3301081D330108AC
:1000F0001D3301081D3301081D3301081D3301089C
:100100001D3301081D3301081D3301081D3301088B
:10011000112101081D3301081D3301081D33010899
:100120001D3301081D3301081D3301081D3301086B
:100130001D3301081D3301081D3301081D3301085B
:100140001D3301081D3301081D3301081D3301084B
:100150001D3301081D3301081D3301081D3301083B
:100160001D3301081D3301081D3301081D3301082B
:100170001D3301081D3301081D3301080000000074
:080180001D3301081D330108C5
:10019000044B05481B1A062B02D9044B03B1184720
:1001A000704700BF8F0000208C000020000000007E
:1001B00005490648091A891001EBD171491002D08E
:1001C000034B03B1184770478C0000208C000020BF
:1001D0000000000010B5064C237843B9FFF7D8FFA4
:1001E000044B13B10448AFF300800123237010BD0A
:1001F0008C000020000000002033010808B5084BE7
:100200001BB108490848AFF300800848036813B9D8
:10021000BDE80840CCE7064B002BF9D09847F7E73C
:100220000000000090000020203301088C00002016
:100230000000000070B50F4E0F4D761BB61018BFB2
:10024000002405D0013455F8043B9847A642F9D163
:100250000A4E0B4D761B03F063F8B61018BF00244E
:1002600006D0013455F8043B9847A642F9D170BD39
:1002700070BD00BF1434010814340108183401089B
:100280001434010870B4860746D0541E002A41D0A9
:10029000CAB2034602E014F1FF343BD303F8012B4A
:1002A0009D07F8D1032C2ED9CDB245EA05250F2C98
:1002B00045EA054519D903F110022646103E0F2ED6
:1002C00042F8105C42F80C5C42F8085C42F8045CAE
:1002D00002F11002F2D8A4F1100222F00F0204F091
:1002E0000F041032032C13440DD91E462246043A43
:1002F000032A46F8045BFAD8221F22F003020432D4
:10030000134404F003042CB1C9B21C4403F8011BCC
:100310009C42FBD170BC704714460346C2E700BF45
:100320000EB410B5044683B018B183690BB900F060
:100330001FF906A803460190059AA168204600F01F
:1003400023FA03B0BDE8104003B070470FB410B5F6
:100350000A4B1C6882B024B1A36913B9204600F08F
:1003600007F905A803460190049AA168204600F009
:100370000BFA02B0BDE8104004B070470000002046
:1003800000207047014900F039B900BFB9110108D8
:100390000020704770B54A1E682505FB02F50E4621
:1003A00005F1740100F054F9044640B100210C300D
:1003B000666005F168022160A060FFF763FF2046D8
:1003C00070BD00BF204B70B51D68AB6906465BB3BE
:1003D00048356B68AC68013B05D521E0013B5A1CF0
:1003E00004F168041CD0B4F90C20002AF6D10025D1
:1003F0004FF6FF720123E281A38165662560A56047
:10040000656025616561A5612946082204F15C00EB
:10041000FFF738FF6563A563A564E564204670BDFA
:10042000286828B10546D4E7284600F00FF8CFE742
:1004300004213046FFF7AEFF28600028F2D10C23DC
:1004400004463360EAE700BF383301083D4B3E49BC
:100450001A682DE9F04F90424FF000038364C364A3
:10046000036508BF012383B008BF8361816207462B
:10047000FFF7A8FF78603846FFF7A4FFB86038465A
:10048000FFF7A0FF7D68F86000240423AB812C6097
:100490006C60AC606C66EC812C616C61AC61214677
:1004A00005F15C000822FFF7EDFEBE68DFF89CB0A6
:1004B000DFF89CA0DFF89C90DFF89C80C5F824B0A2
:1004C00001230922C5F828A0C5F82C90C5F8308072
:1004D0002D622146F381B28134607460B460746629
:1004E00034617461B46106F15C0008220193FFF786
:1004F000C9FEFD68366212200222C6F824B0C6F892
:1005000028A0C6F82C90C6F830802146A881EA8140
:100510002C606C60AC606C662C616C61AC6105F148
:100520005C000822FFF7AEFE019B2D62C5F824B0E7
:10053000C5F828A0C5F82C90C5F83080BB6103B081
:10054000BDE8F08F3833010885030108FD0D01086F
:10055000250E0108610E0108810E0108024B0349B6
:10056000186800F04BB800BF38330108B911010812
:10057000836903B96AE77047704700BF704700BFDF
:10058000704700BF704700BF024B0349186800F076
:100590000FB800BF0000002091030108024B03497F
:1005A000186800F005B800BF0000002081030108B2
:1005B0002DE9F04110F148071BD0884600267D68E0
:1005C000BC68013D0FD4A389012B05F1FF3506D985
:1005D000B4F90E300133204601D0C04706436B1CEE
:1005E00004F16804EFD13F68002FE8D13046BDE840
:1005F000F0813E463046BDE8F08100BF2DE9F8436A
:1006000010F148071FD0884606464FF000097D6864
:10061000BC68013D11D4A389012B05F1FF3508D930
:10062000B4F90E3001332146304602D0C04749EAC2
:1006300000096B1C04F16804EDD13F68002FE6D17E
:100640004846BDE8F883B9464846BDE8F88300BF90
:1006500070B5CC1C24F0030408340C2C38BF0C24D7
:10066000002C06463BDBA14239D8274D296851B101
:100670000A68121B04D436E01A68121B1AD51946F0
:100680004B68002BF8D16968002937D021463046E5
:1006900000F0A2FB431C22D0C31C23F00305A84298
:1006A00005D0291A304600F097FB013017D02C6096
:1006B0002B4604E00B2A0DD91A6013441C6003F189
:1006C0000B0020F007001A1D821A02D051429950E7
:1006D00070BD70BD8B420ED05A684A60EFE70C23A4
:1006E0003360002070BD0B2A03D84A680B462A608D
:1006F000E5E70B46E0E70A460B46F8E7304600F030
:100700006BFB6860C2E700BFA80000209368013B54
:10071000002B10B4936008DBCCB21368581C106037
:10072000197020465DF8044B70479469A34202DBC0
:10073000CCB20A2CF1D15DF8044B00F0A5BB00BF90
:1007400093B1F8B514460F460646D51801E0AC4201
:1007500008D03A4614F8011B3046FFF7D7FF431C78
:10076000F5D1F8BD0020F8BD00207047936810B5A2
:10077000144613B95360184610BD00F061FD002304
:10078000A360636010BD00BF2DE9F04F9DB08946A6
:1007900014460393824618B18369002B00F00A8146
:1007A0008A4B994500F00C81894B994500F00B81EB
:1007B000884B994508BFDAF80C90B9F80C30180747
:1007C00040F1EE80D9F81030002B00F0E9803023A2
:1007D0008DF82A302378804E0021202209918DF84F
:1007E00029200127002B00F08480252B254603D1EA
:1007F00017E0252B00F0858015F8013F002BF8D17C
:10080000B5EB040B75D022465B4649465046FFF7D0
:1008100097FF01306DD0099B2A785B440993002A29
:1008200067D000234FF0FF320135049307930693FE
:100830008DF853301A93059204E0049A07FA03F3F3
:100840001343049329780522304600F0F9FE2C4624
:10085000831B01350028F0D1049BD90644BF202218
:100860008DF8532021781A0744BF2B228DF853208E
:100870002A2969D0A1F13002092A0BD8079B14F864
:10088000011F03EB830302EB4303A1F13002092AAA
:10089000F5D907932E293FD0504D0322284600F06A
:1008A000CFFE38B1049B401B402202FA00F0034304
:1008B0000134049321784A488DF828100622013427
:1008C00000F0BEFE002849D0464BF3B103AB0093C5
:1008D0004A46454B04A95046AFF300808046B8F124
:1008E000FF3F06D0099B434409932378002B7FF4F4
:1008F0007CAFB9F80C305B0659D409981DB0BDE83F
:10090000F08FB5EB040B8CD07DE7039B073323F00E
:10091000070308330393E5E761782A2904F101000E
:1009200026D0A1F130020023092A05930446B3D84A
:1009300014F8011F03EB830302EB4303A1F1300220
:10094000092AF5D90593A7E7039A1168043200290B
:1009500003921FDB0791617801349BE703AB00939F
:100960004A46214B04A9504600F0E6F88046B6E717
:10097000039B1A680592002A03F104030393B8BF8E
:100980004FF0FF3204F10203AEBFA178A1780592C7
:100990001C4681E7494243F0020307910493DAE7DA
:1009A0004946504600F0E8FA00283FF410AF4FF0F7
:1009B000FF30A3E7FFF7DCFD044B99457FF4F4AE6D
:1009C000DAF80490F9E6DAF80890F6E67C330108E4
:1009D0005C3301083C330108D8330108E0330108D7
:1009E000E4330108000000004107010810B4044C82
:1009F00013460A46014620685DF8044BFFF7C4BE63
:100A0000000000202DE9F0470C4691460A698968EC
:100A1000DDF820808A42B8BF0A46C9F8002094F861
:100A2000431006461F4611B10132C9F80020236861
:100A300099065DD5D9F800200232C9F80020236854
:100A400013F0060F19461DD1E1688A1A002AD8BF93
:100A5000194617DD04F1190A002505E0E368D9F805
:100A600000209B1AAB420CDD01235246394630462A
:100A7000C047013005F10105F0D14FF0FF30BDE86E
:100A8000F087216894F84330003318BF01238A06A9
:100A90000AD5E1185A1C302081F84300224494F80A
:100AA000451082F84310023304F1430239463046C0
:100AB000C0470130E1D0236803F00603042B29D09E
:100AC000A36822699342C8BF4FF0000930DD9B1A2A
:100AD00099441A34002501E04D4529D001232246CE
:100AE00039463046C047013005F10105F4D1C4E76D
:100AF00013F0060F08D1E168D9F800208A1A002AFD
:100B0000D8BF1946A6DCBDE794F84330003318BFC0
:100B10000123C9E7D9F80010E068A3682269A0EBB7
:100B20000109934229EAE979D1DCB9F1000FD0D16A
:100B30000020BDE8F08700BF2DE9F0430C46097E98
:100B400085B06E29064617460C98984604F1430C6A
:100B500055D00FD8632900F01B8100F2D680002900
:100B60005CD0582940F0E88084F845102268DFF80E
:100B700060E213E0732900F0FD8000F289806F29A4
:100B800000F0E480702940F0D780226842F0200213
:100B900022607823DFF83CE284F8453003681506CC
:100BA00003F1040100F1FF8055064BBF1B881B6851
:100BB00001600160D00744BF42F020022260002B98
:100BC00040F09580226822F020022260102100224D
:100BD00084F843206068A0600028C0F28D802268FD
:100BE00022F004022260002B67D1002840F08680AA
:100BF000654608296FD0ACEB0503236111E023683B
:100C00001A0600F1D38013F0400F0368626903F104
:100C1000040101601B6814BF1A801A600023654636
:100C20002361CDF800803B4603AA21463046FFF7FA
:100C3000E9FE013021D02A46236939463046C047B3
:100C400001301AD02368E06813F0020F039B19D01B
:100C5000C21A002A16DD04F11909002504E0E06833
:100C6000039BC21AAA420DDD01234A46394630468B
:100C7000C047013005F10105F1D14FF0FF3005B05B
:100C8000BDE8F0839842B8BF184605B0BDE8F083D0
:100C900075295BD078294FD122687AE76168A16015
:100CA0002D200029C3F1000384F8430021DB22F04A
:100CB0000402DFF81CE122600A216546B3FBF1F271
:100CC00001FB123013461EF8002005F8012D002B01
:100CD000F4D108298FD12368D9078CD5626823699C
:100CE0009A4288DC302305F8013C013D83E710215E
:100CF0006DE7DFF8DCE00A21002BDED19EF8003042
:100D000084F8423004F1420573E7642901D069296F
:100D100012D122680368150603F1040152D4550666
:100D20004BBFB3F900301B6801600160002BB5DBDD
:100D3000DFF89CE00A214DE7012384F8421023618B
:100D400004F14205002384F843306AE723681A0659
:100D500033D413F0400F036803F1040215BF1B885E
:100D60001B68026002606F2914BF0A210821DFF8A6
:100D700060E02CE703686268191D01601D680021AE
:100D8000284600F05DFC00B3401B60602061D9E79D
:100D900003681A68191D0123016004F1420584F8F3
:100DA00042202361CEE701601B6803E703686269A4
:100DB000191D01601B681A6030E703681A1D026084
:100DC0001B68D0E701601B68B0E76068DEE700BF22
:100DD000EC3301080034010838B5074C0023054600
:100DE0000846236000F058FE431C00D038BD23683D
:100DF000002BFBD02B6038BD9801002010B50C46AD
:100E0000B1F90E1000F0DAFD002803DB636D034436
:100E1000636510BDA38923F48053A38110BD00BF77
:100E2000002070472DE9F0411646B1F90C201F460D
:100E3000D3050C46054607D500220223B1F90E1052
:100E400000F076FBB4F90C20B4F90E1022F48052B5
:100E5000A2813B4632462846BDE8F04100F076B814
:100E600010B50C46B1F90E1000F062FBA389421CCC
:100E70000EBF23F4805343F480536065A38110BDFB
:100E8000B1F90E1000F0F2B8F8B50D46144606465A
:100E900010B18369002B42D0254B9C4244D0254B96
:100EA0009C4243D0244B9C4208BFF468A389A269AA
:100EB000A2601A0722D5236903B322686169D31A95
:100EC000EDB28B422F4621DA0133A168501C013963
:100ED000A1602060157062699A4206D0A389DB0781
:100EE00001D50A2D01D03846F8BD2146304600F024
:100EF00063F90028F7D04FF0FF37F4E7214630467A
:100F000000F03AF80028F6D12369D6E721463046AA
:100F100000F052F90028EED122680123D5E7FFF74F
:100F200027FB034B9C42BAD17468BFE7B468BDE7A6
:100F30007C3301085C3301083C330108024B0A464C
:100F400001461868FFF7A0BF0000002070B50D46ED
:100F5000084C114606461A4628460023236000F036
:100F6000A9FD431C00D070BD2368002BFBD033606B
:100F700070BD00BF98010020384B70B51D68064653
:100F80000C4615B1AB69002B42D0354B9C4245D085
:100F9000344B9C4258D0344B9C4208BFEC68B4F9A7
:100FA0000C2093B219070CD52069A8B113F00102E7
:100FB0001ED0636900225B42A361A260F0B10020F1
:100FC00070BDDD0642D558072AD4206942F00803D7
:100FD000A3819BB20028E9D103F42072B2F5007F0F
:100FE000E4D03046214600F0E7FAA3892069DDE726
:100FF000990758BF6269A2600028E0D1B4F90C30AB
:101000001A06DDD543F04003A3814FF0FF3070BDD9
:101010002846FFF7ADFA124B9C42B9D16C68BEE787
:10102000616B51B104F14403994204D0304600F0A1
:1010300055FCB4F90C20002363630023206963602E
:1010400022F024022060C1E7AC68A8E742F0400229
:10105000092333604FF0FF30A28170BD00000020F3
:101060007C3301085C3301083C33010838B5074C78
:10107000002305460846236000F0E6FC431C00D030
:1010800038BD2368002BFBD02B6038BD98010020B1
:101090008B891A072DE9F0410D46804633D44A6802
:1010A000002A67DDEC6A002C45D00022D8F80060E9
:1010B000C8F8002013F4805260D06A6D5F0705D530
:1010C00069686B6B521A0BB12B6CD21A0023296A18
:1010D0004046A047441C39D0AB892A692A60DB040A
:1010E0004FF000026A6043D4696BC8F8006011B326
:1010F00005F14403994202D0404600F0EFFB002086
:101100006863BDE8F0810E69AEB10C680E609807A7
:101110000CBF4B690023A41B8B600AE023463246B8
:10112000AF6A296A4046B8470028A4EB0004064489
:1011300004DD002CF2DC0020BDE8F081AB8943F037
:101140004003AB814FF0FF30BDE8F081D8F80020BC
:101150001D2AF3D8174BD340DB4313F00103EDD125
:10116000A9892C696B60C9042C60BDD5002ABBD14C
:101170006865B9E70A6C002A94DCDCE70123296A78
:101180004046A047431C024602D0AB89EC6A95E773
:10119000D8F80030002BF8D01D2B01D0162B02D12F
:1011A000C8F80060C7E7AB8943F04003AB81BDE8F6
:1011B000F08100BF010040200B6933B310B5044635
:1011C00082B008B18369ABB1114B994219D0114B70
:1011D000994218D0104B994208BFE168B1F90C3020
:1011E00013B9002002B010BD204602B0BDE8104087
:1011F000FFF74EBF0191FFF7BBF90199044B9942EC
:10120000E5D16168EAE7A168E8E70020704700BF20
:101210007C3301085C3301083C33010820B1054BE5
:1012200001461868FFF7C8BF034B04491868FFF769
:10123000E5B900BF0000002038330108B9110108EA
:101240009368002B73D02DE9F04F8B8983B00C4647
:1012500019070090164626D5226922B313F0020022
:1012600035682CD04FF00009B04FC846B246B8459B
:1012700043464A4628BF3B460098B8F1000F50D07D
:10128000216AA66AB047002858DDDAF808301B1A30
:101290008144A8EB0008CAF80830002BE7D10020F1
:1012A00003B0BDE8F08F21460098FFF765FE0028E7
:1012B00040F03381A389356813F00200D2D113F0D6
:1012C000010945D14F46019637B39A05D4F80880F5
:1012D00040F183804745C346C0F0AB8013F4906F64
:1012E00040F0AC802068BA465A46494600F092FA6F
:1012F000A2682368A2EB08025B44A2602360019A03
:101300009368A3EB0A03D144A7EB0A079360002B71
:10131000C5D0A389002FD8D1D5F800906F680835C3
:10132000D2E7D5F80090D5F8048008359FE7002073
:10133000704721460098FFF73FFF70B3B4F90C30B7
:1013400043F040034FF0FF30A38103B0BDE8F08FBE
:10135000814633464E46A8469A464D464EB380B324
:10136000206823696269B145CB4628BFB3469842DD
:101370005F4604D9A36813449B4500F3A6809345B8
:101380004BDB1346A76A216A00982A46B847071E16
:10139000D4DDB9EB0709CCD00120DAF80830DB1B2B
:1013A0003D44F61BCAF80830002B3FF478AF002EFE
:1013B000D5D108F1080313E9600098460833002EE0
:1013C000F9D032460A21284600F03AF9002800F008
:1013D000A1800130A0EB0509C2E72068236998428B
:1013E00002D863699F425DD2B84528BFB8464246DD
:1013F000494600F00FFAA3682268A3EB08034244B1
:10140000A36022600BB1C24679E721460098FFF73E
:10141000D3FE002892D1C24671E75A46294600F011
:10142000F9F9A2682368A2EB0B025B44A260236077
:10143000AFE72068B846BA46BB4655E76269206800
:10144000216902EB4208A0EB010A08EBD8780AF107
:1014500001004FEA680838444045424684BF804650
:1014600042465B0544D511460098FFF7F1F88346E4
:10147000002855D05246216900F032F9A38923F49F
:10148000906343F08003A3810BEB0A00A8EB0A03EF
:10149000C4F810B0C4F814802060A360B846BA46FF
:1014A000BB4621E76FF00041B94228BF39464A46A2
:1014B00091FBF3F10098A66A03FB01F3216AB047A0
:1014C000B0F1000A3FF71BAF38E71A4629460193EF
:1014D00000F0A0F92268019B00981A44226021467E
:1014E000FFF76AFE019B00287FF428AF1F4650E7F4
:1014F000009800F03BFA83460028C5D1009D216981
:10150000284600F0EBF9B4F90C300C2223F08003EC
:101510002A6015E706F1010922E74FF0FF30BFE628
:10152000009A0C231360B4F90C3009E700FCFF7F2C
:1015300070B50D46084C114606461A46284600234B
:10154000236000F099FA431C00D070BD2368002B83
:10155000FBD0336070BD00BF9801002070B50C4611
:10156000B1F90E10002990B015461E4613DB01AAF2
:1015700000F03AFA00280EDB029A02F47042A2F55B
:101580000052B2FA82F252094FF4806300203260B6
:101590002B6010B070BDA38900221B06326004D5F9
:1015A000402300202B6010B070BD4FF480630020FA
:1015B0002B6010B070BD00BF8A8992070B4606D51C
:1015C00001F1470201211A601A6159617047F0B5B3
:1015D00083B001AB6A460C460546FFF7BFFF009992
:1015E00006462846FFF734F8B4F90C30D0B1019A1A
:1015F000124F0099AF6243F08003A3812060206105
:1016000061611AB93343A38103B0F0BD2846B4F930
:101610000E1000F0FDF9B4F90C300028F2D043F0C0
:101620000103EFE79A05EFD404F1470243F0020308
:101630000121A381226022616161E5E78503010840
:1016400001F0FF01102A2BDB10F0070F08D010F873
:10165000013B013A8B422DD010F0070F42B3F6D177
:10166000F0B441EA012141EA014122F007047FF090
:1016700000070023F0E80256083C85EA010586EAE7
:10168000010685FA47F5A3FA87F586FA47F6A5FA23
:1016900087F68EB9EED1F0BC01F0FF0102F007022F
:1016A00032B110F8013B013A83EA010313B1F8D1DA
:1016B0000020704701387047002D06BF35460338BB
:1016C000073815F0010F07D1013015F4807F02BFF4
:1016D000013015F4C03F0130F0BC0138704700BF45
:1016E000844641EA000313F003036DD1403A41D32D
:1016F00051F8043B40F8043B51F8043B40F8043BEC
:1017000051F8043B40F8043B51F8043B40F8043BDB
:1017100051F8043B40F8043B51F8043B40F8043BCB
:1017200051F8043B40F8043B51F8043B40F8043BBB
:1017300051F8043B40F8043B51F8043B40F8043BAB
:1017400051F8043B40F8043B51F8043B40F8043B9B
:1017500051F8043B40F8043B51F8043B40F8043B8B
:1017600051F8043B40F8043B51F8043B40F8043B7B
:10177000403ABDD2303211D351F8043B40F8043B1B
:1017800051F8043B40F8043B51F8043B40F8043B5B
:1017900051F8043B40F8043B103AEDD20C3205D32B
:1017A00051F8043B40F8043B043AF9D2043208D023
:1017B000D2071CBF11F8013B00F8013B01D30B8895
:1017C00003806046704700BF082A13D38B078DD073
:1017D00010F003038AD0C3F10403D21ADB071CBF45
:1017E00011F8013B00F8013B80D331F8023B20F8AF
:1017F000023B7BE7043AD9D3013A11F8013B00F8E8
:10180000013BF9D20B7803704B7843708B7883706F
:10181000604670478842F0B50DD98B1898420AD2BD
:101820008418002A51D0224613F8014D02F8014DC8
:101830009942F9D1F0BD0F2A48D941EA00039B072C
:1018400046D100F1100401F11003154653F8106C55
:1018500044F8106C53F80C6C44F80C6C53F8086C9A
:1018600044F8086C103D53F8046C44F8046C0F2DD8
:1018700003F1100304F11004E8D8A2F1100323F0DF
:101880000F0302F00F0E1033BEF1030F194403448F
:1018900021D91E1F0D467446043C55F8047B46F8BA
:1018A000047F032CF8D8AEF1040424F003040434BC
:1018B0002144234402F0030262B1013B0A4411F8BF
:1018C000014B03F8014F8A42F9D1F0BD0346F3E71B
:1018D0000346F2E7F0BD7246EEE700BF91B151F862
:1018E000043C0439002BB8BFC9181F4B1A68FAB161
:1018F0008A4230B40AD908680C18A24226D04A603D
:10190000196030BC70478B4203D81A465368002BCD
:10191000F9D1146815198D420DD006D808680C1835
:101920009C4219D04B605160EBE70C230360E8E761
:101930004A601960704709680C4411199942146093
:10194000DFD10ACB0C4453601460DAE714685268A4
:101950004A6020440860D3E71C685B684B60204401
:1019600008605160CDE700BFA8000020F8B514461C
:10197000F9B1C2B106460D4600F05CF8844201D8C8
:101980002846F8BD21463046FEF762FE074670B194
:1019900022462946FFF7A4FE294630463D46FFF77A
:1019A0009DFF2846F8BDFFF799FF2546E8E7054665
:1019B000E6E71146BDE8F840FEF74ABE70B50D46B1
:1019C000084C114606461A4628460023236000F0BC
:1019D0005BF8431C00D070BD2368002BFBD0336044
:1019E00070BD00BF9801002038B50B46074C054676
:1019F000114618460023236000F02EF8431C00D047
:101A000038BD2368002BFBD02B6038BD9801002027
:101A100038B5074C002305460846236000F024F83B
:101A2000431C00D038BD2368002BFBD02B6038BD91
:101A30009801002051F8040C0028A0F10400BCBF5C
:101A40000B58C018704700BF024B58221A604FF065
:101A5000FF30704798010020024B58221A604FF067
:101A6000FF30704798010020024B58221A60002076
:101A7000704700BF98010020024B58221A604FF0B7
:101A8000FF30704798010020024B58221A604FF037
:101A9000FF30704798010020044A05491368002B65
:101AA00008BF0B461844106018467047B00000206D
:101AB000A001002070B595B214460E462A464FF696
:101AC000FF73064800F036FD2A4631464FF6FF7395
:101AD000034800F02FFD204670BD00BF1401002018
:101AE00054010020DFED187A184AB5EEC00A20EE46
:101AF000270AF1EE10FA70B501464FF06405FDEECD
:101B0000C07A0DD417EE903A82FB0302DC17C4EBC7
:101B1000621205FB12330E48BDE87040FEF716BC9A
:101B200017EE904A604282FB0036C31782FB04E244
:101B3000C3EB6613E41705FB1303C4EB62120448FE
:101B4000BDE87040FEF702BC0000C8421F85EB51A3
:101B50009C330108F0B595B008A830220021FEF7AB
:101B600091FB00241D4A0194049403940594069467
:101B70000794116C1A4B41F080511164126C02F001
:101B800080520192019A02941A6842F480421A60CB
:101B90001B680F9403F4804302930123022508215C
:101BA00048220B9308A80323102610911192139337
:101BB000029F08950E9512950C9600F08FFE0F224D
:101BC0004FF4805303A82946049505940794039283
:101BD000069301F079F815B0F0BD00BF003802405F
:101BE0000070004000B587B000230D4A00930193B8
:101BF0000393029304930593136B43F01003136351
:101C0000136B019003F01003009301A90223054810
:101C1000009A039301F040F907B05DF804FB00BFA0
:101C2000003802400004024008B54FF48060FFF71E
:101C3000D9FF4FF48061104801F044FA01280DD01B
:101C40000E4B0F489FED0F0A00221A60FFF74AFF64
:101C500042F21070BDE8084001F002BB074902469D
:101C60000A2309480A6000F065FC42F21070BDE8E2
:101C7000084001F0F5BA00BF00100240B400002097
:101C8000A83301080000000014010020414B424A23
:101C9000424C80B59A6001F0BBFAFFF75BFF00F0A1
:101CA00097F800F06BF900F031F900F04BF90A23D6
:101CB00005223B493B4800F03DFC4FF47A7001F0AF
:101CC000CFFA0A2305223849364800F033FC214672
:101CD0004FF4FA631422334800F088FC0A231422DC
:101CE0002146324800F026FCA37C5A1E012A49D91D
:101CF000052B05D10A230B222D492C4800F01AFC94
:101D00002C4C2D4F2D4EDFF8C0802D4DFFF78CFF52
:101D100023680F2BFADC384600224FF4806101F073
:101D2000D7F9384600224FF4807101F0D1F93046DE
:101D300000224FF4004101F0CBF9304600224FF46D
:101D4000005101F0C5F9304600224FF4006101F066
:101D5000BFF9404600224FF4004101F0B9F928468E
:101D600000224FF4004101F0B3F9284600224FF45D
:101D7000005101F0ADF900224FF40061284601F056
:101D8000A7F9C3E70A2307220E49084800F0D2FB4F
:101D9000B6E700BF00ED00E000000108C000002031
:101DA0006C00002054010020640000201401002079
:101DB0007C000020B400002000000240000C024023
:101DC000001002407400002000040240704700BF71
:101DD0002DE9F0438BB00024464B00941A6B464D1E
:101DE000DFF82091DFF82081444F454E42F0010298
:101DF0001A631A6B02F001020092009A01941A6BA6
:101E000042F010021A631A6B02F010020192019A5A
:101E100002941A6B42F002021A631A6B02F0020279
:101E20000292029A03941A6B42F008021A631A6B28
:101E300002F008020392039A04941A6B42F004021F
:101E40001A631B6B03F004030493284601224FF42A
:101E50007841049B01F03CF9484601224FF440418F
:101E600001F036F9404601224FF47C4101F030F98F
:101E7000384601224FF4007101F02AF90122304660
:101E80004FF47C5101F024F9284605A901254FF4AF
:101E90007843059307940894069500F0FDFF4846A3
:101EA00005A94FF44043059306950794089400F064
:101EB000F3FF404605A94FF47C430593069507942C
:101EC000089400F0E9FF384605A94FF40073059324
:101ED00006950794089400F0DFFF4FF47C5305A9A2
:101EE0003046069507940894059300F0D5FF0BB093
:101EF000BDE8F083003802400010024000080240B4
:101F00000000024000040240000C02400B4B0C4A4F
:101F100010B50C211A604FF4E134002218465C60C1
:101F200059619A60DA601A619A61DA6100F0D2FA56
:101F300000B910BDBDE81040FFF748BF14010020F4
:101F4000004C00400B4B0C4A10B50C211A604FF4AA
:101F5000E134002218465C6059619A60DA601A61C7
:101F60009A61DA6100F0B6FA00B910BDBDE8104020
:101F7000FFF72CBFD4000020001001400B4B0C4A8F
:101F800010B50C211A604FF41644002218465C600C
:101F900059619A60DA601A619A61DA6100F09AFA1E
:101FA00000B910BDBDE81040FFF710BF540100207C
:101FB00000440040F0B503683C4A934289B02BD0FE
:101FC0003B4A93424DD03B4A934201D009B0F0BD09
:101FD0000024394B0294196C384841F400311964DB
:101FE0001B6C03F4003302930322072303A9602729
:101FF00002260125DDF808E0069207930397049670
:10200000059500F049FF22462146262001F088F878
:10201000262001F0BBF8D9E70024274B0094196C67
:10202000274841F4002119641B6C03F4002300933A
:102030000322082303A94FF4406702260125DDF897
:1020400000E00692079303970496059500F024FF9D
:1020500022462146342001F063F8342001F096F83E
:10206000B4E70024144B0194596C164841F0100158
:1020700059645B6C03F0100301930322072303A947
:10208000C02702260125DDF804E006920793039796
:102090000496059500F000FF22462146252001F018
:1020A0003FF8252001F072F890E700BF004C004097
:1020B000001001400044004000380240000C024083
:1020C0000008024000040240704700BFFEE700BF66
:1020D000FEE700BFFEE700BFFEE700BF704700BF9E
:1020E000704700BF704700BF08B501F0ABF8BDE80E
:1020F000084001F073B800BF014800F021BB00BFE9
:10210000D4000020014800F01BBB00BF5401002098
:10211000014800F015BB00BF1401002008B50320E2
:1021200000F0ECFF002211466FF00B0000F0F8FF0A
:10213000002211466FF00A0000F0F2FF0022114663
:102140006FF0090000F0ECFF002211466FF0040070
:1021500000F0E6FF002211466FF0030000F0E0FF00
:10216000002211466FF0010000F0DAFF0022114654
:102170004FF0FF30BDE8084000F0D2BF2DE9F04736
:10218000046822698246C068DAF81C10DAF8083060
:10219000DAF81060DAF8145022F440520243226157
:1021A000E268DAF81800334322F416422B4322F097
:1021B0000C020B431343E360636923F4407303434E
:1021C000B1F5004F6361AB4B61D09C4200F00181DF
:1021D00003F580639C4200F0FC8000F02DFEA64FCA
:1021E000DAF8043000EB800000EB80009B00B0FBCD
:1021F000F3F3A7FB03235B091D0100F01DFEDAF8D2
:10220000043000EB80009B0000EB8000B0FBF3F695
:1022100000F012FEDAF8042000EB8000930000EBDF
:102220008000B0FBF3F3A7FB03234FF064095B09C5
:1022300009FB13631B013233A7FB03235B0903F084
:10224000F00600F0F9FDDAF8042000EB80009300BE
:1022500000EB8000B0FBF3F800F0EEFDDAF804309C
:1022600000EB80009B0000EB8000B0FBF3F0A7FBCD
:102270000030400909FB10831B013233A7FB032305
:10228000C3F3431333432B44A360BDE8F0879C4260
:102290005DD003F580639C4259D000F0CDFD764FB0
:1022A000DAF8043000EB800000EB80005B00B0FB4C
:1022B000F3F3A7FB03235B091E0100F0BDFDDAF871
:1022C000043000EB80005B0000EB8000B0FBF3F516
:1022D00000F0B2FDDAF8042000EB8000530000EBC0
:1022E0008000B0FBF3F3A7FB03235B094FF0640905
:1022F00009FB1353DB003233A7FB03231B0903F451
:10230000F87500F099FDDAF8042000EB800000EB8E
:1023100080005300B0FBF3F800F08EFDDAF80430D3
:1023200000EB800000EB80005B00B0FBF3F3A7FB49
:1023300003235B0909FB1383DB003233A7FB032371
:10234000C3F3421333442B44A360BDE8F08700F08D
:102350008BFD494FDAF8043000EB800000EB800081
:102360005B00B0FBF3F3A7FB03235B091E0100F046
:102370007BFDDAF8043000EB80005B0000EB8000AE
:10238000B0FBF3F500F070FDDAF8042000EB8000FC
:10239000530000EB8000B0FBF3F3A7FB03234FF0E7
:1023A00064095B0909FB1353DB003233A7FB0323EA
:1023B0001B0903F4F87500F057FDDAF8042000EB70
:1023C0008000530000EB8000B0FBF3F800F04CFD00
:1023D000A4E700F049FD284FDAF8043000EB800054
:1023E00000EB80009B00B0FBF3F3A7FB03235B092A
:1023F0001D0100F039FDDAF8043000EB80009B008D
:1024000000EB8000B0FBF3F600F02EFDDAF80420BC
:1024100000EB8000930000EB8000B0FBF3F3A7FB20
:1024200003234FF064095B0909FB13631B0132337B
:10243000A7FB03235B0903F0F00600F015FDDAF8B3
:10244000042000EB8000930000EB8000B0FBF3F869
:1024500000F00AFDDAF8043000EB800000EB8000A9
:102460009B00B0FBF3F3A7FB03235B0909FB13837A
:1024700002E700BF001001401F85EB512DE9F0413C
:1024800007460E4690461D463C6801E06B1C06D18F
:10249000206836EA0003F9D10020BDE8F08135B1AB
:1024A00000F0D8FEA0EB08008542EDD23C68E3685E
:1024B00023F4D073E3606369202223F00103002139
:1024C0006361032087F8392087F8381087F83A20AD
:1024D000BDE8F08160B338B590F83930044603F0B8
:1024E000FF0203B32268242384F83930D36823F42D
:1024F0000053D3602046FFF741FE23681A6922F497
:1025000090421A615A6922F02A025A61DA6800255B
:10251000202142F40052DA602846E56384F839103D
:1025200084F83A1038BD80F83820FFF743FDD9E72A
:10253000012070472DE9F0430F4690F8391020290B
:1025400083B003D0022003B0BDE8F083002F3ED05B
:10255000002A3CD0984690F83830012B0446F1D040
:10256000002001212123E06384F8381084F83930F9
:10257000019200F06FFE019AA2848146E28406E097
:10258000FFF77CFF28BB23683A785A600137E58C57
:10259000ADB243464A4680212046E5B1E58CA668A7
:1025A000013DADB2B6F5805FE584E9D143464A46C8
:1025B00080212046FFF762FF58B93B8821682269D5
:1025C000C3F308034B60002AE0D10237DFE70120A4
:1025D000B9E70320B7E74021FFF750FF0028F8D103
:1025E000202384F8380084F83930ACE72DE9F04333
:1025F0000E4690F83A10202983B003D0022003B091
:10260000BDE8F08376B36AB3984690F83830012B72
:102610000446F3D0002001212223E06384F838101F
:1026200084F83A30019200F015FE019AA2858146A5
:10263000E285E58DADB243464A462021204685B36A
:10264000E58DA768013DADB2B7F5805FE58512D095
:10265000FFF714FF58BB236933B923685B683370F5
:102660000136E6E70120CAE723685B6803F07F03D1
:1026700033700136DDE743464A4620212046FFF706
:10268000FDFEA0B9236933B923685B68C3F308036F
:1026900026F8023BCDE723685B68DBB226F8013BF6
:1026A000C7E784F83850284684F83A10A7E7032093
:1026B000A5E700BF704700BF704700BF8368B3F550
:1026C000805F28D0036973B10368826A5B68511C1C
:1026D00003F07F0381621370C38D013B9BB2C385FE
:1026E00043B100207047836A0268591C52688162B6
:1026F0001A70F1E70268D16821F4907110B5D160C9
:102700005169202421F00101516180F83A40FFF71E
:10271000D3FF002010BD0269836A3AB9026852688B
:10272000C2F3080223F8022B8362D5E702685268DD
:10273000D2B223F8012B8362CEE700BF704700BFFF
:1027400003681A6870B51607DD685969044649D0F0
:1027500011F0010152D0D60705D5E80503D5E06B8D
:1027600040F00100E06356077AD5002900F084802C
:10277000E16B900741F00201E16376D5E16B41F036
:102780000401E163110772D4E16B002929D091069D
:1027900005D5AA0603D594F83A20222A7CD05D6993
:1027A000E16B0E0702D415F040057AD0DA6822F406
:1027B0009072DA605A69202122F001025A6184F88D
:1027C0003A105A6955065ED55A69606B22F040028C
:1027D0005A61002857D03B4B036500F07DFC002870
:1027E00055D170BD96060CD5A9060AD590F83A3099
:1027F000222BF6D1BDE87040FFF760BF15F4907F43
:10280000A9D110060ED45606EBD56D06E9D5DA68C7
:10281000202122F04002DA60204684F83910FFF7C8
:1028200049FF70BD2906EED594F83920212AD8D168
:10283000A268B2F5805F226A38D0511C21621278FA
:102840005A60E28C013A92B2E284002AC9D1DA6875
:1028500022F08002DA60DA6842F04002DA6070BD8D
:1028600096070BD5002989D18EE711078CD5E16B2E
:1028700041F00801E16387E7900785D4100783D50D
:10288000002981D0F3E72046FFF758FF70BD606B49
:10289000BDE87040036D18472046FFF70FFF23681F
:1028A0007DE72046FFF74AFFE56370BD1188206988
:1028B000C1F30801596010B902322262C1E7013246
:1028C0002262BEE7C928010808B5836B0022DA85B9
:1028D0001846DA84FFF732FF08BD00BFF0B5036881
:1028E000DD0783B004462FD5A3498A6802F00C02A5
:1028F000042A00F0F4808A6802F00C02082A00F032
:10290000EA806368B3F5803F00F02C81B3F5A02F17
:1029100000F00081984D2A6822F480322A602A68EB
:1029200022F480222A60002B40F0FD8000F092FC0F
:10293000064605E000F08EFC801B642800F2AA80A9
:102940002B689B03F6D423689F072DD58A4A91688C
:1029500011F00C0F00F0A580916801F00C0108291E
:1029600000F09B80E368002B00F0EB80834B824DEE
:1029700001221A6000F06EFC064605E000F06AFCD9
:10298000801B022800F286802B689807F6D52968FC
:10299000F82292FAA2F22369B2FA82F221F0F80147
:1029A00093400B432B6023681A0720D4590734D473
:1029B000A369CBB1704DAA6802F00C02082A77D047
:1029C000022B6F4B4FF000021A6000F0D18000F034
:1029D00041FC2C46054604E000F03CFC401B02286C
:1029E00058D823689B01F7D4002003B0F0BD636979
:1029F000002B60D0634B604D01221A6000F02AFC6E
:102A0000064604E000F026FC801B022842D86B6FCB
:102A10009F07F7D523685907CAD5574B5A4D00224F
:102A200001921A6C42F080521A641B6C03F08053BE
:102A30000193019B2B6843F480732B6000F00AFC28
:102A4000064604E000F006FC801B022822D82B6812
:102A5000DA05F7D5A368012B00F0F180052B00F013
:102A6000D580454D2A6F22F001022A672A6F22F095
:102A700004022A67002B40F0D28000F0EBFB41F209
:102A8000883607462B6F980792D500F0E3FBC01BF2
:102A9000B042F7D9032003B0F0BD526856023FF5AB
:102AA00061AF354A1268950723D5E268012A20D024
:102AB000012003B0F0BD334A2F4D136000F0CAFB74
:102AC000064604E000F0C6FB801B0228E2D86B6FCC
:102AD0009807F7D49EE74A6850027FF512AF264A5E
:102AE000126891037FF530AF6268002A7FF42CAF43
:102AF000DEE7214DF821286891FAA1F12269B1FAA7
:102B000081F120F0F8008A4002432A601A077FF51D
:102B10004DAF6CE7184B1A6842F480221A601A68AD
:102B200042F480321A6000F095FB134D064604E033
:102B300000F090FB801B6428ACD82B689A03F7D573
:102B400001E70E4A0C4D136000F084FB064604E0DA
:102B500000F080FB801B02289CD82B689907F7D4D3
:102B6000236821E7044A136843F480331360DAE7EB
:102B700000F070FB06460FE00038024000004742BC
:102B800060004742800E47420070004000F062FB48
:102B9000801B02283FF67EAF2B689901F6D447F6DA
:102BA000C07696FAA6F64FF44032B6FA86F692FA56
:102BB000A2F24FF07061B2FA82F091FAA1F1A26A2A
:102BC000676AE369D4F820E0E46A520843EA0E0336
:102BD00007FA06F6013A8240B1FA81F1334304FA6A
:102BE00001F11343194A1A4C0B4301216B60116028
:102BF00000F030FB054605E000F02CFB401B0228EE
:102C00003FF648AF23689A01F6D5EDE6104B1A6FF0
:102C100042F004021A671A6F42F001021A6700F0CC
:102C200019FB0B4D074641F288362B6F9B073FF58A
:102C3000BFAE00F00FFBC01BB042F6D92AE7044A32
:102C4000136F43F001031367E9E700BF60004742D9
:102C500000380240194A936803F00C03042B2BD070
:102C6000082B27D15168536801F03F0113F4800FFE
:102C7000536847F6C07292FAA2F0B0FA80F003EA05
:102C8000020323FA00F314BF0D480E48B0FBF1F025
:102C900000FB03F0094B4FF440325B6892FAA2F25A
:102CA000B2FA82F203F44033D34001335B00B0FB4D
:102CB000F3F07047034870470148704700380240FE
:102CC00040787D010024F400574A136803F00F0395
:102CD0008B4208D2CBB21370136803F00F039942F2
:102CE00001D00120704703689A072DE9F04106D50D
:102CF0004E4C8568A26822F0F0022A43A260DF07EA
:102D000006460C4626D54268012A00F08780931EAD
:102D1000012B464B1B687BD9990728D5434DAB68DF
:102D200023F003031343AB6000F094FA7368012BA4
:102D3000074641F288384FD0022B58D0032B05D1DB
:102D400060E000F087FAC01B404564D8AB6813F020
:102D50000C0FF6D1344A136803F00F039C4209D2DA
:102D6000E3B21370136803F00F039C4202D00120FA
:102D7000BDE8F08133685A0706D52C49F0688A68A7
:102D800022F4E05202438A601B0707D5274A3169C3
:102D9000936823F4604343EAC1039360FFF75AFF4B
:102DA000224B0146F0229B6892FAA2F2B2FA82F21A
:102DB00003F0F003D3401E481E4AC35C002021FAF2
:102DC00003F3136000F00EFA0020BDE8F08100F07C
:102DD00041FAC01B40451ED8AB6803F00C03042B1E
:102DE000F5D1B7E700F036FAC01B404513D8AB6801
:102DF00003F00C03082BF5D1ACE700F02BFAC01B55
:102E0000404508D8AB6803F00C030C2BF5D1A1E7C3
:102E1000980183D4ABE70320BDE8F081034B1B6826
:102E20009D033FF57BAFA2E7003C02400038024023
:102E3000C433010888000020084B4FF4E0529B681F
:102E400092FAA2F2B2FA82F203F4E053D3400449B8
:102E5000044ACB5C1068D840704700BF003802407D
:102E6000C433010888000020084B4FF460429B687F
:102E700092FAA2F2B2FA82F203F46043D340044918
:102E8000044ACB5C1068D840704700BF003802404D
:102E9000C4330108880000202DE9F04FD1F800C0AC
:102EA000DFF81482DFF814E283B0002503E0013577
:102EB000102D00F09B800123AB4003EA0C029342EB
:102EC000F5D14E6826F0100ABAF1020F00F0918099
:102ED0004FEA45090324D0F800B004FA09F4E443AA
:102EE00006F003070BEA040B07FA09F70AF1FF3AA9
:102EF00047EA0B07BAF1010F076040F2A080C768EC
:102F00008B683C4003FA09F32343C360F300CED53A
:102F10004FF00009CDF80490D8F8443043F48043D2
:102F2000C8F84430D8F8444025F0030303F1804347
:102F300004F4804403F59C33019405F00304019FDD
:102F4000D3F808A0A4000F27A7402AEA070A544F85
:102F5000B84222D007F58067B84200F08380514F15
:102F6000B84200F08480504FB84200F085804F4F47
:102F7000B84200F086804E4FB84200F087804D4F37
:102F8000B84200F08880DFF8389148450CBF4FF018
:102F900007094FF0080909FA04F94AEA09079F608E
:102FA000DEF80030D443F70354BF23401343CEF878
:102FB0000030DEF80430B70354BF23401343CEF88B
:102FC0000430DEF80830F70254BF23401343CEF834
:102FD0000830DEF80C30B60205F1010554BF23407D
:102FE0001343102DCEF80C307FF465AF03B0BDE86D
:102FF000F08F4FEAD50900EB890905F00707D9F8EA
:103000002040BF004FF00F0B0BFA07FB24EA0B0A1E
:103010000C69BC4044EA0A04C9F820404FEA45095B
:103020000324D0F800A004FA09F4E44306F00307EF
:103030000AEA040A07FA09F747EA0A0707608768F5
:1030400007EA040ACF6807FA09F747EA0A07876020
:10305000D0F804A0C6F300172AEA0303AF401F43C9
:1030600047604CE74FF0010909FA04F995E74FF082
:10307000020909FA04F990E74FF0030909FA04F983
:103080008BE74FF0040909FA04F986E74FF00509C8
:1030900009FA04F981E74FF0060909FA04F97CE717
:1030A0000000024000080240000C024000100240F4
:1030B000001402400018024000380240003C014069
:1030C000001C02400369194214BF01200020704710
:1030D00002B909048161704790F83530022B03D0A2
:1030E00080234365012070470268052380F835304E
:1030F000136823F00103136000207047074AD36868
:103100004FF6FF010B40000243F0BF6300F4E060A4
:1031100043F400330343D360704700BF00ED00E089
:10312000184B70B4DC68C4F30224C4F10706042E03
:1031300004F1040328BF0426062B17D9033C0125FC
:10314000A540013D2A400123B340013B1940A14065
:10315000002841EA02010CDB00F1604000F561400B
:103160000901C9B280F8001370BC704700221446F0
:10317000E9E7054B00F00F0009010344C9B21976D5
:1031800070BC704700ED00E0FCEC00E000F01F01B7
:1031900001234009024A8B4042F82030704700BFAB
:1031A00000E100E00138B0F1807F0ED2084B10B48E
:1031B000084C5860F02084F82300002207211046B4
:1031C0009A6019605DF8044B70470120704700BF9A
:1031D00010E000E000ED00E0704700BF08B5FFF729
:1031E000FBFF08BD084B094A1B6810B5A2FB03236F
:1031F00004469809FFF7D6FF214600224FF0FF3022
:10320000FFF78EFF002010BD88000020D34D621014
:1032100008B50B4B1A6842F400721A601A6842F43F
:1032200080621A601A6842F480721A600320FFF705
:1032300065FF0020FFF7D6FFFEF770FF002008BDF6
:10324000003C0240024A136801331360704700BF1C
:1032500094010020014B1868704700BF94010020C2
:1032600010B582B00190FFF7F5FF0446FFF7F2FFBB
:10327000019B001B9842F9D302B010BD1049114BBD
:10328000D1F8882042F4700210B4C1F888201A687E
:103290000D4C002042F001021A6098601A6822F07A
:1032A000847222F480321A605C601A684FF0006405
:1032B00022F480221A60D8608C605DF8044B70475D
:1032C00000ED00E00038024010300024DFF834D078
:1032D000002103E00C4B5B58435004310B480C4B6E
:1032E00042189A42F6D30B4A02E0002342F8043B0C
:1032F000094B9A42F9D3FFF7C1FFFCF79BFFFEF79A
:10330000C5FC7047000002201C34010800000020AA
:103310008C0000208C0000209C010020FEE70000B3
:10332000F8B500BFF8BC08BC9E467047F8B500BFB2
:08333000F8BC08BC9E46704782
:103338000400002000000000000000000000000061
:103348000000000000000000000000000000000075
:103358000000000000000000000000000000000065
:103368000000000000000000000000000000000055
:103378000000000000000000000000000000000045
:103388000000000000000000000000000000000035
:10339800000000002573203D2025642E25640A00C6
:1033A8004D31395F627574746572666C7976616CDB
:1033B8007665666565646261636B00000000000005
:1033C8000102030401020304060708094300000080
:1033D800232D302B20000000686C4C006566674583
:1033E80046470000303132333435363738394142B8
:1033F8004344454600000000303132333435363717
:0C340800383961626364656600000000F2
:04341400FD010108AD
:04341800D5010108D1
:10341C0004000020000000007C3301085C3301082C
:10342C003C33010800000000000000000000000018
:10343C0000000000D4330108000000000000000070
:10344C000000000000000000000000000000000070
:10345C000000000000000000000000000000000060
:10346C000000000000000000000000000000000050
:10347C0000000000FE00010001000000FE00020040
:10348C0002000000636F6E6E656374006E6F7420D3
:0C349C00636F6E6E656374000024F40022
:04000005080132CDEF
:00000001FF
